:020000020000FC
:100000006DCEC1C10000000020C000008EC0000005
:10001000000098C000000000000000000203040679
:10002000080C10182030406080000406080C1018DE
:100030002030406080A0C0000003070F1F000D0D9E
:100040000403060D0503030202004FB662FD0CC057
:10005000552041F00994C52DC095089483FDC7959E
:10006000C4BD64604FBE1895C0916400089483FDC0
:10007000C795C4BD6B7FC0916400CF3F09F41EC01B
:1000800070FF1AC082FD05C04FBE9798AC98959836
:10009000189576FD0EC064FD0CC0C091B100C0FD86
:1000A000AB98C1FDAD98C2FD9498CAEFC095CA95B2
:1000B000F1F79798AC9895984FBE189524BCCC272B
:1000C000C064C8BF6460F8CFC6CF70FFC4CF64FD02
:1000D000C2CF979AC0CF70FFBECF64FDBCCFAC9AA1
:1000E000BACF70FFB8CF64FDB6CF959AB4CFAB9AB4
:1000F00070FFB1CF64FDAFCFC7E0CA95F1F7979A13
:10010000AACFAD9A70FFA7CF64FDA5CFC7E0CA956F
:10011000F1F7AC9AA0CF949A70FF9DCF64FD9BCF6E
:10012000C7E0CA95F1F7959A96CF4FB6C9B7CF7E7B
:10013000C9BF6E7FCCB5CE0DDDB5DF1DDBBDCABD41
:100140004FBE18953FB68F7EABB7A074A2118061E9
:10015000A0E0ABBFA9B7AE7FA9BF7894A09168001B
:10016000AA2341F085FD2EC0A0916800AA95A09316
:10017000680028C040E050E085FD14C0A0B396FDA3
:10018000A095A2FD4FEFA3E096FDA2E0A5BFAA2790
:10019000A064AABF8D7FA0B396FDA095A2FD5FEFDE
:1001A000451741F7A0E461FDA093680085FD03C0F9
:1001B000A0E4A0936800409396008160442311F06E
:1001C0002092990085FD0EC0A0916900AA2331F00C
:1001D000A0916900AA95A093690004C08061AA2734
:1001E000A064AABF80FF0AC0A09196004A2F61FFB9
:1001F0008E7F85FD01C000C0409361004091B40036
:10020000443009F004C0A0916100A0936300A09164
:100210006000A395A093600051F0F894A9B7A16085
:10022000A9BF84FF02C0A0E4ABBF3FBE1895A09158
:100230007400A395A093740042E050916800552388
:1002400029F085FF03C05A9550936800A09196004D
:10025000A13018F0209299000DC020929A002092AF
:10026000A300A0919900AF5FA093990018F0AFEFA1
:10027000A0939900B09061005091B400523049F4BD
:1002800065FF91F0A2E3BA1678F0A0918600A093E2
:100290006100533049F465FF39F0A2E3BA1620F04B
:1002A000A091C000A0936100509162005B1521F005
:1002B00010F05A9501C05395509362004A95D1F6BB
:1002C0005091A300539509F45A955093A300A0911F
:1002D000A400AA95A093A40009F04BC0A1E0A093AC
:1002E000A40048E0A091A500AA2381F145E0A091D7
:1002F000A5005A17F0F1A091A6005A1728F441E082
:10030000A3E0A093A40007C0A091A7005A1718F477
:1003100041E04093A400D0909C00C0906300DC14A6
:10032000A8F0A091B400A430D9F065FD0FC0C09230
:100330009C00539521F0A091A500A093A300A1E0FB
:10034000A093A400ACE3A093620013C0A0919C0012
:10035000A40F20F45FEF50939C0002C0A0939C0078
:10036000A0919C00AF3F29F4AFEFA0939A00A09317
:10037000A300F894A9B7A160A9BF84FF02C0A0E4BC
:10038000ABBF3FBE18953FB64CB55DB58F7EABB7E2
:10039000A074A2118061A0E0ABBFA9B7AE7FA9BFD6
:1003A000789481FD23C0A2E096FDA3E0A5BF826002
:1003B000A0B396FDA095A2FF05C0409365005093A1
:1003C00066001CC1A3E096FDA2E0A5BFAA27A06419
:1003D000AABF8D7F85FF01C004C140E0A0B396FD98
:1003E000A095A2FDFEC040939600EDC0A3E096FD4F
:1003F000A2E0A5BF8D7F61FF71C0A2E096FDA3E0E2
:10040000A5BFAA27A064AABF826040939100509321
:100410009200A0908F004A19B09090005B09BB2415
:10042000A22C4C38520518F42092950049C0A09196
:10043000D400AA2359F1483C520528F4A0E1BA2E71
:10044000AAE0AA2E23C04836A1E05A0728F4A8E063
:10045000BA2EAFE0AA2E1AC0403DA2E05A0728F4F7
:10046000A4E0BA2EAEE1AA2E11C0403AA5E05A0788
:1004700028F4A2E0BA2EACE3AA2E08C04839A8E0BE
:100480005A0720F4A1E0BA2EA8E7AA2EC42EA09104
:100490009300CA1AD52EA0919400DA0ADD202AF41E
:1004A000AFEFC094D094CA1ADA0A20929500A8E05F
:1004B000A210A0E0CA14DA0618F4A1E0A0939500F7
:1004C000409393005093940040919100509192007A
:1004D00040938F005093900042E075C0A09165005A
:1004E0004A1BA09166005A0B94FD60C093FD5EC04C
:1004F00092FD5AC086FF03C0D52EC42E0CC056955F
:10050000479591FD51C05695479590FD4DC0D52E0C
:10051000C42ED694C79461FD19C0AC2DAC51AD2D3D
:10052000A24008F005C0DD2089F4AC2DA85C70F471
:10053000A0916700A395AA2311F0A0936700AA30A9
:1005400008F44FC02092960081604BC0A0916700D4
:10055000AA2319F0AA95A0936700A22C5091BA0083
:1005600097FD02C0A090C800AAEFAA0EA22DA21D5E
:10057000CA18DA0A4FB74170442319F040E050E03E
:1005800015C0AFEFCA16D20418F04FEF50E00EC0FE
:10059000A091AC00CA9E412D000C441F50E008F011
:1005A00012C04FEF50E00FC05695479594FF07C01B
:1005B000552309F04FEFA42FA6954A0F521D4F3F28
:1005C000520508F04FEF40939600816061FF09C02B
:1005D000AFE1A095A923AB299A2F8F7DBB2009F409
:1005E0008062A0E4A093680085FF03C0AAE0A09306
:1005F000680061FD03C085FD01C08F7E85FD03C0DD
:10060000A0E2A0936900F894A9B7A160A9BF84FFF4
:1006100002C0A0E4ABBF3FBE189511E00AC013E0D2
:1006200008C01AE006C01EE104C014E602C018ECBF
:1006300000C005E1BB27BA95F1F70A95D9F71A95DD
:10064000C1F708952AE338E709C020E33CE806C073
:100650002AE234EB03C025E238EC00C0B091AD00D3
:10066000BA9509F4089512E0BB27AD9ABA95F1F74F
:10067000AC9ABA95F1F7AC98BA95F1F7AD98BA95EE
:10068000F1F7123009F0979A123009F4959AB09167
:10069000AD00BA95F1F7123009F09798123009F4CD
:1006A0009598B7E8BA95F1F71A95F1F6022FB22F9F
:1006B000BA95F1F70A95D9F73A9581F6AD9A08956A
:1006C000221B39E0001F3A9509F40895221F211BCF
:1006D00018F4210F8894F6CF0894F4CF622C722C72
:1006E000B0E08894B395221F331FE0F73795279524
:1006F0008894912E802E020B130B10F4192D082DC7
:1007000010F4889401C00894661C771CBA9571F7A0
:10071000172D062D0895322D11232AF43A950095B0
:100720001095031B130BF894029F712C002D129F40
:10073000912C802C7894780C172D921C292DB4E0E4
:100740006B2E2695179507956A94D9F7332321F0D8
:1007500000951095031B130B08950091B40004300D
:1007600009F474C0B0919600B95198F0B72FB670E3
:1007700081F465FD2BC005E09090C600B92DBA95B7
:1007800021F00AE0BA9509F002E1B0917B00B01BBC
:10079000E0F065FF0AC0B0919E00B0939C00BFEFEF
:1007A000B093A300B1E0B093A400B0916100B09306
:1007B000630020927E0020927F0020928000209291
:1007C0008100209282006F7D41C060629090C600DF
:1007D000B92DBA9579F4B0916200B095BB1FBB1FDB
:1007E0001B2FB7950B2FB12FB170B3951B2FB02FC7
:1007F000BE7F25C0B92DBA95BA9581F4B09162003B
:10080000B095BB1FBB1FBB1F1B2FB7950B2FB12F65
:10081000B370B3951B2FB02FBC7F14C0B091620092
:10082000B095BB1FBB1FBB1FBB1F1B2FB7950B2F4B
:10083000B12FB770B395B3951B2FB02FB87FB054BD
:100840000B2F120900937E0010937F0008951091E2
:100850007B00169500917A000795B0917E00B01B41
:100860000B2FB0917F00B10B1B2F28F40038BFEF86
:100870001B0740F009C00F37120508F405C00FE749
:1008800010E002C000E81FEF009383001093840083
:10089000089500918300B09180000B0F10918400A7
:1008A000B09181001B1F20E03091840033230AF4B3
:1008B0002A95B09182002B1F1AF4203F40F00AC005
:1008C0002F3008F407C00FEF1FEF2FE003C000E048
:1008D00010E020EF30916300B0919B003B1718F4BB
:1008E000323030F009C0B0918400BB235AF004C00C
:1008F000B0918400BB2332F40093800010938100F8
:100900002093820008952091D70000918300000F6A
:1009100010918400111FFFDE11232AF40038BFEF6D
:100920001B0740F009C00F37120508F405C00FE798
:1009300010E002C000E81FEF002352F0B091620007
:10094000B01B0B2F18F0013008F00AC001E008C0FE
:1009500000950F5FB09162000B0F08F001C00FEF20
:100960000093850008952091D80000918100109196
:100970008200D1DE11232AF40130BFEF1B0740F0C3
:1009800009C00F3F120508F405C00FEF10E002C0C8
:1009900001E01FEF112352F0B0918500B01B0B2F27
:1009A00018F0013008F00AC001E008C000950F5FA0
:1009B000B09185000B0F08F001C00FEF00936300AA
:1009C00008950FEF71FD1EC0B091D300BB23D1F08D
:1009D000B0917B00BB23B1F00FEF10917B0070DE74
:1009E000F894B091730072FDB5E00B9F112D002DAE
:1009F0007894112309F00FEFB0919E000B1710F4BB
:100A000000919E0000939D00089500917A0010913E
:100A10007B0000541140B0919D0010F4BA9501C0C4
:100A2000B39511F0B0939D000895EBD3B1E074FD40
:100A3000B2E0B7B9B6B1B068B064B6B9EEDDB1E056
:100A400074FDB2E0B7B9B6B1B068B064B6B9B6B1CA
:100A5000B6FDFDCF04B115B1B6B1BF77B6B928D494
:100A600027E32093A800222309F441C030E030930B
:100A7000A900732E7694622E6694620E731E262D44
:100A8000372D0217130778F08090A800B7E3B80D50
:100A9000B093A8008090A900B0E0B81DB093A90061
:100AA000260D371DEECF8090A8009090A9001091E0
:100AB000A90016950091A80007951695079523E0C3
:100AC000169507952A95E1F72091B5002A9529F406
:100AD0002092A8002092A9000AC02A9521F0800E39
:100AE000911E2A95E1F78092A8009092A90008959E
:100AF0002091B500B6B1B6FDFBCF04B115B1B6B1CA
:100B0000BF77B6B9B091AA00B395B093AA00B83038
:100B100060F12092AA00B091D200BB2321F11123F1
:100B200029F0B091AB00BF3F61F009C0B091AB00BC
:100B30000B1739F020F4BB2321F0BA9502C0B3950E
:100B4000E1F300919B00B093AB00B33650F400EC9E
:100B5000BB3538F400E8B33520F400E4BB3408F4C6
:100B600000E000939B007F7E08952130B1F00F3F9D
:100B7000B3E01B0790F4B7E3BB2379F0B091A80072
:100B80000B17B091A9001B0740F4B0919B00BB2349
:100B900059F0BA95B0939B0007C0B0919B00BF3F3E
:100BA00019F0B395B0939B0000919B00B091630046
:100BB000B01B10F400916300B0919C000B1750F033
:100BC00000919C00B0919C00BF3F21F0B0919C002F
:100BD000B0939B00502E00936400B091AA00B730F0
:100BE00009F47061089502E3F894B091D9000B9F65
:100BF000012D000C001F7894B0919B000B1710F092
:100C000000919B000093610000936300502E0093BD
:100C1000640000939E00089520927A00B0EFB09394
:100C20007B000895F8940CB51DB52091740078945C
:100C300030917500609076000093750010937600F7
:100C4000031B160971FD03C077FD80C028C070909A
:100C50007700209377002709222319F00FEF1FEF69
:100C60000EC0809078009090790030937800609268
:100C700079000091750010917600081919092091EA
:100C80007A0030917B0036952795020F131F10F4E0
:100C90000FEF1FEF00937A0010937B002BC0209181
:100CA0007A0030917B003901B4E08B2EB2E09B2EAC
:100CB000343040F08A949A94383020F072FD02C0AB
:100CC0008A949A94769467948A94E1F7261937095E
:100CD000992021F0169507959A94E1F7200F311F7E
:100CE00020937A0030937B0028F43FEF30937A0012
:100CF00030937B00323008F4706871FF02C0B3E0BB
:100D00000DC0B091C40000917100023838F0B39565
:100D1000003A08F0B395B63008F0B5E09B2EB4E089
:100D20008B2E10917B0000917A0024E01695079598
:100D30002A95E1F70819120928F0B02FB250B12F07
:100D4000B20910F402E010E0980126C020917A0068
:100D500030917B003901769467946694669466942A
:100D60002619320906950695200F321D20937A0028
:100D700030937B00323008F07F7704E0369527957A
:100D80003695279526952695201B10F0223008F4DD
:100D900022E089019090C40060FDFECFE0908B00BE
:100DA000F0908C006160B9B7B061B9BF380177FDD0
:100DB00041C07694679400938B0010938C00B92DFA
:100DC000B330E1F0B0FD04C0060D171D930106C05D
:100DD000000F111F0250120922E030E0B92DB3308C
:100DE00068F020938D0030938E000093870010935D
:100DF00088006092890070928A003AC000938D004A
:100E000010938E00209387003093880060928900B1
:100E100070928A0071FF0DC0BFE0B0938D002092E8
:100E20008E00B093890020928A00B0938B002092AC
:100E30008C001EC0669400938B00B92DB33091F0E6
:100E4000B0FD03C0060D262D03C0000F025022E0A6
:100E5000B92DB33038F020938D0000938700609255
:100E6000890006C000938D0020938700609289005E
:100E700000917C0002FD0350013029F495FD0AC069
:100E8000B0E0B7B909C0023019F4B7E0B7B904C08F
:100E900095FDF6CFB6E0B7B90091A200000F10F4AF
:100EA000BBE60B270093A20060FDFECFB2E0B0933B
:100EB0006E006160B9B7B061B9BFB72FB670D1F03D
:100EC00020917A0030917B003695279536952795AD
:100ED00071FF02C0B0E43B0FF8940CB51DB5020FD2
:100EE000131F1BBD0ABD6160B0E1B8BFB9B7B061E7
:100EF000B9BF78940895686020927D0020E066FD77
:100F000020E206C0686020927D0020E266FD20E0BD
:100F100001E011E077FD11C0B72FB67009F0677FCF
:100F200014E100917B00069509F403950F3008F059
:100F30000FE071FF02C004E114E160FD0FC0B09149
:100F40007D00BB2359F071FF06C0B0916E00BA95C9
:100F5000B0936E0011F470624FC0ABDFB0B7B77FD3
:100F6000B0BFB8B1B0B7B860B0BFB0917D00B395B5
:100F7000B0937D00B8B177FD06C0B1E071FDB3E07C
:100F8000BA95F1F7B8B1B072B21709F02AC071FF83
:100F900005C00395011708F00A95CFCF63FD05C082
:100FA0000395011708F0B4CFC8CF677FF8943CB51C
:100FB0006DB470907A00B0917B00770CBB1F08F481
:100FC000BFEF770CBB1F08F4BFEF370D6B1E6BBC78
:100FD0003ABD6160B0E1B8BFB9B7B061B9BF78944C
:100FE00097CFB0916D00B13008F492CF63FD90CFF0
:100FF0000A9509F0A2CF7F7D20918D0030918E005F
:10100000F894B0E1B8BF0CB51DB5020F131F1BBD9E
:101010000ABDE0908700F09088006160B9B7B061C8
:10102000B9BF7894B72FB67039F0B0916D0072FFE8
:10103000B395B0936D0009C075FF07C066FD05C08C
:1010400063FD03C0BF91BF91F4C4089500E063FF46
:1010500001C001E0F89410917100B7E01B9F212DB1
:10106000102D7894200F269517952695179526957F
:10107000179510937100183718F4B8E7B093710002
:1010800000917100B09172000B1720F06061979889
:10109000AC98959860FDFECFE0908900F0908A00B2
:1010A0006160B9B7B061B9BF0895B2E095FD0AC0FB
:1010B000F894B0937C00AD9AAB9862FF01C0959A0A
:1010C0007894F4C0F894B0937C00AD9A949862FF41
:1010D00001C0979A7894EAC0B3E082FF24C095FDDE
:1010E00011C002E0F894B0937C00E1E8F0E00093D6
:1010F000B1009598949A62FF02C0AC9A01C0AD9875
:101100007894D4C002E0F894B0937C00E1E8F0E079
:101110000093B1009798AB9A62FF02C0AC9A01C0ED
:10112000AD987894C3C095FD0BC0F894B0937C0043
:10113000EBE6F0E0959862FF01C0AC9A7894B6C0F7
:10114000F894B0937C00EBE6F0E0979862FF01C062
:10115000AC9A7894ABC0B4E095FD0AC0F894B09313
:101160007C00AB9A949862FF01C0AC9A78949EC0C0
:10117000F894B0937C00949AAB9862FF01C0AC9A4B
:10118000789494C0B5E082FF24C095FD11C001E0C1
:10119000F894B0937C00E7E7F0E00093B100AC98DE
:1011A000AD9A62FF02C0979A01C0AB9878947EC056
:1011B00004E0F894B0937C00EBE8F0E00093B10019
:1011C000AC98AD9A62FF02C0959A01C09498789449
:1011D0006DC095FD0BC0F894B0937C00E5E6F0E09F
:1011E000AC9862FF01C0979A789460C0F894B0936D
:1011F0007C00E1E7F0E0AC9862FF01C0959A78943A
:1012000055C0B6E095FD0AC0F894B0937C00949A5E
:10121000AD9862FF01C0979A789448C0F894B09353
:101220007C00AB9AAD9862FF01C0959A78943EC05D
:10123000B1E082FF24C095FD11C004E0F894B093A2
:101240007C00EBE8F0E00093B1009798AB9A62FF66
:1012500002C0959A01C09498789428C001E0F8944F
:10126000B0937C00E7E7F0E00093B1009598949A82
:1012700062FF02C0979A01C0AB98789417C095FDA1
:101280000BC0F894B0937C00E1E7F0E0979862FF20
:1012900001C0959A78940AC0F894B0937C00E5E672
:1012A000F0E0959862FF01C0979A78946F7E089558
:1012B00024E630E0F9012092B1009798AC98959817
:1012C000AB9AAD9A949A6B7F0895A2EBB0E007E0D9
:1012D0000D9307E00D9301E00D9304E00D930FEFE4
:1012E0000D930D9309E00D9302E00D9301E00D9332
:1012F00001E00D93AEEBB0E001E00D9300E00D9343
:1013000004EB0D930FEF0D930D930D9303E00D93ED
:101310000FEF0D9301E00D930FEF0D9305E20D9389
:1013200000ED0D9308E70D9308EC0D9304E00D9389
:101330000FEF0D9301E00D9300E00D930AE70D937D
:101340000AE00D9300E00D9301E00D9300E00D9392
:101350000FEF0D9300E00D9308952091B9008B7F5E
:10136000233009F48460B091BA009F7DB1FD906292
:101370009F7BB091BB00B1FD9064223011F088607A
:1013800001C0877F08950A95E00FF21DB49108957A
:10139000ECE1F0E00091B200F6DFB093D700ECE1B1
:1013A000F0E00091B300EFDFB093D800EAE2F0E0A4
:1013B0000091B800E8DFB093D9000091D10000237C
:1013C00019F42092A50013C0013108F001E1B02FFB
:1013D000B00FB00FB093A5001B2FB10FB10FB00F1E
:1013E000B093A600B10FB00FB00FB093A70000915B
:1013F000B800023008F402E000937300B091CE0010
:101400000FEFB23009F400EAB33009F402E80093B8
:101410007200E8E3F0E00091D500B5DFB093A000E2
:10142000089508952091C8003091C900B091BA0084
:10143000B33009F43E5097FF02C020E03FEFB32FD6
:10144000B21B6B2EB25810F4B2E86B2E00E003957D
:10145000609EB12DBD57D8F30093AC0008959068FD
:10146000E1DFE1D8E0D820E030E0B0E16B2ED7D862
:10147000B09196002B0F321D6A94C9F7B4E03695EF
:101480002795BA95E1F7822E9F77CCDF0895F894DF
:10149000E3E0F0E0B9E0B7BFB491B078C1F3F894FD
:1014A000A895B1B5B861B1BDB0E0B1BDB4E0BEBF03
:1014B000BFE5BDBFFDDEB0E0B8BBB0E1B7BBB8E291
:1014C000B5BBB8E3B4BBB0E1B2BBB0EBB1BB222457
:1014D000A0E0B0E02D92AA31E9F7A0E6B0E00FEF6E
:1014E0002D920A95E9F7B1E0B093A200EEDEDED2CC
:1014F000B6B1B460B6B90091CA000093AD00B1E0D6
:10150000B0936A00F89493D89DD88DD89ED88BD884
:101510009FD889D85AD38BD88AD887D8F8940AEF1D
:101520001AEFA0B396FDA095A2FF1FC01A95C9F7A8
:101530000A95B1F7E0E0FCE1B591B43E39F4B5911C
:10154000B03E21F4B591BF3F09F40CC0E0E0F39543
:10155000F395B591B83F49F4B591B43931F4B591EB
:10156000BA3A19F4EE27F6950994F7DE11DF59DF40
:1015700059DF0091CA000093AD009ADEB2E0B3BF1C
:10158000B2E0BEBDB2E0B5BDB1E5B8BFB9BFB0B75E
:10159000B77FB0BFB8B1B0B7B860B0BF3ED878942D
:1015A00044DA20927000B3E096FDB2E0B5BFB0E43B
:1015B000BBBFBB27B064BABF8D7F39D8626033E050
:1015C0002CE0B0919500BB2321F42CE03A9509F46E
:1015D000A5CF29D880FFA2CF8E7FB0919600B230E0
:1015E00078F3B92FBF710091980000939700B093E2
:1015F0009800B01729F72A9521F76D7FB3E096FD83
:10160000B2E0B5BFBB27B064BABF8D7FB091D40044
:10161000BB2321F48062B92FB0709B2F8F7B209267
:10162000670003D885FF05C0B0916700BA3008F0A5
:101630008064F5D702E085FF01C000E0B09196001C
:10164000B017B8F3F894FED7FDD7FCD77894EFD74E
:1016500020928600E4D7B091BE00B13008F478C083
:10166000B0916A00B13008F473C085FD18C0B09124
:101670009600BF3F08F46CC0F894EDD77894D5D7A6
:10168000B0919600B130C0F7F894DCD7CAD7DAD75A
:101690007894CBD7B0919600BF3FB0F3C8C2B8E002
:1016A0009B2E9068F894BEDE7894BFD7F8949F770D
:1016B000B9DE80909600B0919600BF37789408F418
:1016C0004FC0ABD7F894C7D778949A9451F7C7DE38
:1016D000B82DB550B093C900AAD7F8947BD27894AE
:1016E000BAE09B2E9068F8949DDE78949ED7F8948B
:1016F0009F7798DE80909600B0919600BF377894DF
:1017000078F78BD7F8949ED78CD79CD778949A94F7
:1017100049F7A5DEB82DBB5FB093C8000B2F109121
:10172000C900125810F0100B20F4B2E80B0F009310
:10173000C9007DD7F894E7D15CD2789476D7F89435
:1017400071DE7894B0919600BF3F08F48ECF6FC2DF
:1017500000919600B09186000B1710F00093860060
:1017600064D701E0B091BA00B35009F405E0B0913C
:101770009600B01708F06ECFF8946DD76CD76BD782
:10178000789455D720926A0020926B0020926C00CA
:10179000B0916B00B395B0936B00BF3F71F5B09102
:1017A0006C00B395B0936C00B091CC0009E1BA9590
:1017B00059F002E3BA9541F00DE7BA9529F00AEF26
:1017C000BA9511F020926C00B0916C00B017A8F09F
:1017D0006FDD23D7B0916C00BA95B0936C00209266
:1017E0006B00B091CB00B093AD00F89434D77894EF
:1017F000B091CA00B093AD0018D713D7B09168006C
:10180000BB2319F485FF01C089CE01E085FD01C02D
:1018100006E0B0919600B01708F4BACF06D7B091A1
:101820006800BB2309F47ACEF89442DD209261006F
:101830002092620020926300522C20926400209239
:10184000A1007894B091B700BB0FB0939F00209295
:101850007E0020927F0020928000209281002092C2
:1018600082002092AA0060E070E020927100B8E04F
:10187000B093AA007061D1D6B1E074FDB2E0B7B9FF
:10188000B6B1B068B064B6B9B6B1B6FDFDCF04B1BB
:1018900015B1B6B1BF77B6B9112309F00FEF0093B8
:1018A000AB0026D9B8E0B093AA00706156DDF89479
:1018B000BFEFB0939B0097D9B0916100B0939B00AC
:1018C000B0939C00B0939D007894B1E0B093610018
:1018D000B09363005B2EB0936400B093A400B0910A
:1018E0009A00B093A300B091BA00B33019F49F7D71
:1018F00087FD90627160726020926D0082DC98DCDE
:101900008BD990D989D98ED987D9FCDA26D79EDB95
:10191000CCDB88D9F0DA65FD9AD777FF52D877FD0E
:1019200074D894DBD9DB7ED9EDDA65FDB2D78EDBD6
:1019300012DC78D9E0DA65FDE6D788DB23DC72D9E2
:10194000E1DA65FD10D882DB5CDC6CD9D4DAB1E079
:1019500074FDB2E0B7B9B6B1B068B064B6B976DBC1
:1019600067DC60D9C5D871FF1EC0B0919E00B093EE
:101970009B00B0939C00B0919A00B093A300B1E09B
:10198000B093A40018E12CE0B0916D00B11728F0DD
:101990007D7F746020936F0006C0B0919600B130D7
:1019A00008F0B3CF50C072FF15C066FD13C0B091F0
:1019B0006F00BA9519F47B7F7860A7CFB0936F0062
:1019C000B0919600B13008F0A0CFB091BA00B3301A
:1019D00009F039C020927000B0919900B13058F0F0
:1019E000B0919E00B0939C00B0919A00B093A30078
:1019F000B1E0B093A400B09199000AEF1091D60025
:101A0000112309F003E0B01708F01DC085FF04C0E2
:101A1000B0916800BB23B9F000EF66FF05C0B0913C
:101A20009E00B0939B0000E2B0917B00B01708F4D9
:101A30006CCFB0917000B395B0937000B0919600E8
:101A4000BB2309F002C020927000F89431DC809032
:101A5000B900B2E0B093B90080DC8092B900209266
:101A600061002092620020926300522C2092640058
:101A700020929F0060E070E07894D7D519DC009147
:101A8000D600002319F0979AAC9A959AB6B1B46033
:101A9000B6B985FF05C0B0916800BB2309F43ECDFF
:101AA000B091BF00B13008F0C4CD6ECEEDE0F0E0F3
:101AB00023D0053A09F01BC0EEE0F0E01DD00A3556
:101AC00009F015C03AE0A2EBB0E0E3E0F0E014D09A
:101AD0000D9331963A95D9F739E1AEEBB0E0EFE0EE
:101AE000F0E00AD00D9331963A95D9F702C0EDDBBC
:101AF0000AD0E8E2F0E00895E199FECFEEBBFFBB2B
:101B0000E09A0DB308951ED03AE0A2EBB0E0E3E016
:101B1000F0E00D910FD031963A95D9F739E1AEEB5F
:101B2000B0E0EFE0F0E00D9105D031963A95D9F7AD
:101B300012D00895E199FECF0DBBEEBBFFBBE29A38
:101B4000E19A0895EDE0F0E00FEFF4DFEEE0F0E071
:101B50000FEFF0DF0895EDE0F0E005EAEBDFEEE0F7
:101B6000F0E00AE5E7DF08953091AE000091AF00A4
:101B7000313011F40093B200323011F40093B3000D
:101B8000333011F40093B400343011F40093C600E4
:101B9000353011F40093B500363011F40093B800DD
:101BA000373011F40093C400383011F40093B900B9
:101BB000393011F40093CE003A3011F40093BA009A
:101BC0003B3011F40093BB00089525E030D52A95F1
:101BD000E9F7089537D539D53BD53DD522D532D54E
:101BE00034D536D538D51DD52DD52FD531D533D5CE
:101BF000089531D52DD529D525D513D52CD528D562
:101C000024D520D50ED527D523D51FD51BD508958E
:101C10008090AE009090AF0015D514D513D501D5A6
:101C20008A94D1F718D5FDD49A94E1F70895F894E1
:101C3000D1DF7894CADFC9DFB1E0B093AE00B1E084
:101C4000B093AF002092B000F894E2DF7894B5E052
:101C50006B2E70909600EBD4B09196007B16C9F76E
:101C6000B13018F0BF3F40F107C07EDFF8944BDF82
:101C7000B1DFB8E0B1BDA9DF6A9459F7B091B00007
:101C8000B395B093B000B33008F4DECF9EDFB091CF
:101C9000AF00B395B093AF00F894B091AE00BA9591
:101CA000EEE3F0E0EB0FF21D049178940395B09110
:101CB000AF00B01708F4C6CF88DF87DFB091AE0061
:101CC000B395B093AE00B091AE00BC3008F4B7CF7E
:0E1CD000FCDAF89418DFB8E0B1BD77DFD8CBAE
:00000001FF
